:1000000044EF05F00000000000EF00F000000000E9
:0A0010000000000000000000F3D71C
:06001C00000000001200CC
:100022000FEE81F0EF50EFCF00F0009C00C0EFFF29
:020032001200BA
:100034000FEE81F0EF50EFCF00F0009E00C0EFFF15
:020044001200A8
:10004600010E02011A6F000E1B6F800E1C6F000E50
:100056001D6F1C511D1125E0DEDFDDDFDCDFDBDF80
:10006600E6DF939ED8DFD7DF1C511915006E000E10
:100076001D15016E0050011002E0938C02D0CEDFF8
:10008600939CC9DFC8DF938E0101F89181BE04D02D
:10009600F8A101D001D0FAD702011D331C331D9FF0
:1000A600D8D71A6B1B6BB7DFB6DFC1DF939EB3DF02
:1000B600B2DF938CB0DFAFDFAEDFADDF938E010131
:1000C600F89181BE04D0F8A101D001D0FAD702017F
:1000D6001A6B1B6BA0DF9FDF81AC01D01A819BDFFF
:1000E6009ADF99DF98DF97DF96DF95DF94DF93DF5E
:1000F60092DF91DF90DF8FDF8EDF8DDF8CDF97DF82
:0C010600939E8CDF939C1AC200F0120044
:1001120087DF939C82DF81DF938E0101F89181BE9C
:1001220004D0F8A101D001D0FAD777DF76DF75DFEE
:1001320074DF73DF72DF71DF70DF938C6EDF6DDF70
:020142001200A9
:0A014400120E0D6E0D2EFED71200F4
:10014E00938C65DF64DF938E62DF61DF63DF939CE8
:0A015E005EDF5DDF68DF939E120094
:10016800086A096A100E0C6E013408360936045004
:10017800085E0550D8A0053C095ED8B007D00450E9
:1001880008260550D8B0053C0926D8900036013617
:060198000C2EEAD7120054
:0E019E00ACB202D00000FCD719C2ADFF1200B7
:1001AC0019C202F01AC203F002C000F003C001F041
:1001BC00024A032A00C0E9FF01C0EAFFEE5201E047
:1001CC00F3D702011951025C006E1A510358016EEB
:0A01DC00010E005E000E015A120031
:1001E6000B6A0A6A096A086A0E6A033408360450FA
:1001F600085E0550D8A0053C095E0650D8A0063C0E
:100206000A5E0750D8A0073C0B5EE86AD8A0010E2C
:100216000E5E0336070E0C6E0334083609360A36B0
:100226000B360E36045003A012D0085E0550D8A037
:10023600053C095E0650D8A0063C0A5E0750D8A0C9
:10024600073C0B5EE86AD8A0010E0E5E11D00826A8
:100256000550D8B0053C09260650D8B0063C0A26FB
:100266000750D8B0073C0B26E86AD8B0010E0E2618
:1002760003360C2ED1D70234083609360A360B3629
:100286000E36045003A012D0085E0550D8A0053CD7
:10029600095E0650D8A0063C0A5E0750D8A0073C67
:1002A6000B5EE86AD8A0010E0E5E11D00826055036
:1002B600D8B0053C09260650D8B0063C0A26075099
:1002C600D8B0073C0B26E86AD8B0010E0E260236D7
:1002D600070E0C6E0234083609360A360B360E3611
:1002E600045002A012D0085E0550D8A0053C095E55
:1002F6000650D8A0063C0A5E0750D8A0073C0B5E05
:10030600E86AD8A0010E0E5E11D008260550D8B0B6
:10031600053C09260650D8B0063C0A260750D8B038
:10032600073C0B26E86AD8B0010E0E2602360C2EC4
:10033600D1D70134083609360A360B360E36045044
:1003460002A012D0085E0550D8A0053C095E0650F2
:10035600D8A0063C0A5E0750D8A0073C0B5EE86AA8
:10036600D8A0010E0E5E11D008260550D8B0053C67
:1003760009260650D8B0063C0A260750D8B0073CD6
:100386000B26E86AD8B0010E0E260136070E0C6E53
:100396000134083609360A360B360E36045001A0EB
:1003A60012D0085E0550D8A0053C095E0650D8A0BC
:1003B600063C0A5E0750D8A0073C0B5EE86AD8A048
:1003C600010E0E5E11D008260550D8B0053C092650
:1003D6000650D8B0063C0A260750D8B0073C0B2674
:1003E600E86AD8B0010E0E2601360C2ED1D700349D
:1003F600083609360A360B360E36045001A012D0DE
:10040600085E0550D8A0053C095E0650D8A0063CFB
:100416000A5E0750D8A0073C0B5EE86AD8A0010E1A
:100426000E5E11D008260550D8B0053C09260650A8
:10043600D8B0063C0A260750D8B0073C0B26E86A17
:10044600D8B0010E0E260036070E0C6E00340836A4
:1004560009360A360B360E36045000A012D0085E56
:100466000550D8A0053C095E0650D8A0063C0A5E99
:100476000750D8A0073C0B5EE86AD8A0010E0E5EB6
:1004860011D008260550D8B0053C09260650D8B02C
:10049600063C0A260750D8B0073C0B26E86AD8B0B7
:1004A600010E0E2600360C2ED1D700B00ED0045009
:1004B60008260550D8B0053C09260650D8B0063C9B
:0C04C6000A260750D8B0073C0B26120095
:1004D200800E02011B6F000E1C6F1D6B1E6B1B51E9
:1004E2001C111EE09ADD99DD938C97DD96DD938ECB
:1004F2000101F89181BE04D0F8A101D001D0FAD750
:1005020081AC05D002011B511D131C511E130201A7
:1005120084DD83DD8EDD939E1C331B331C9FDFD76E
:10052200938C7BDD7ADD19511A1102E079DD939CFF
:1005320074DD73DD938E0101F89181BE04D0F8A1C0
:1005420001D001D0FAD769DD68DD73DD939E65DDE8
:0C05520064DD66DD939C1DC200F0120009
:10055E000900F5CFE6FF0006FBE10106F9E1120006
:0A056E00000E9EBA010E006E12008E
:100578000201136B050E135D0AE213511125E16E9A
:10058800000E1221E26E200EE66E132BF3D71351E4
:100598001125E16E000E1221E26EE66A130713516F
:1005A8001125146F000E1221156F0A0E046E000E2D
:1005B800056E0FC200F010C201F0D2DD08C000F0D5
:1005C80009C001F0300E002614C2E1FF15C2E2FF97
:1005D80000C0E6FF0A0E046E000E056E0FC200F0A2
:1005E80010C201F0BDDD00C00FF201C010F2000E14
:1005F800011802E1000E001801E102D01307CFD75D
:020608001200DE
:10060A000FC204F010C205F004C0E9FF05C0EAFFFA
:10061A00EE5203E0044A052AF7D704C002F005C0E7
:10062A0003F0044A052A11C200F012C201F00201C5
:10063A00114B122B00C0E9FF01C0EAFF02C0E1FF23
:10064A0003C0E2FFEECFE6FF02C0E9FF03C0EAFF04
:10065A00EE5201E0E2D70FC200F010C201F0120020
:10066A00FF0E816E080E936E806A896A2F0E926E53
:10067A00820EC16E010EC26E826A8B6A946A120081
:10068A00ECC119F2EDC11AF28CDD00C010F20F6B49
:10069A000F510101EC25E96E000E02010FBFFF0E9A
:1006AA000101ED21EA6EEECF19F274DD02010F2B82
:1006BA00800E0F19006E800E1019005CE9E312001B
:1006CA000FC204F010C205F004C002F005C003F026
:1006DA00044A052A11C200F012C201F00201114BAC
:1006EA00122B00C0E9FF01C0EAFF02C0E1FF03C00C
:1006FA00E2FFEECFE6FF02C0E9FF03C0EAFFEE52D7
:0E070A0001E0E2D70FC200F010C201F01200B1
:10071800F00E02010F15026E02C000F00032009EBA
:100728000032009E0032009E0032009E300E0024EF
:10073800016E01C010F20150390802E2070E1027BD
:100748000F0E0F15006E300E0024016E01C011F25D
:100758000150390802E2070E112710C219F21BDDF9
:1007680011C219F218DD680E0201196F14DD1200AA
:100778000D0E0201196F0FDD0A0E0201196F0BDD54
:0207880012005D
:10078A0002010F6B106B116B126B0F0E136F020EBF
:10079A00146F0101FF51800F0201056F00510527F7
:1007AA0006510527CFDC530E0D6E0D2EFED7D00E47
:1007BA00196F44DC530E0D6E0D2EFED705C219F2C9
:1007CA003DDCA2DCBFDCD10E0201196F37DC030E5F
:1007DA001325E16E000E1421E26EE66A020E13255D
:1007EA00156F000E1421166F010E196F000E1A6F85
:1007FA006BDE030E001615C2E1FF16C2E2FF00C04F
:10080A00E6FF010E02011325156F000E1421166F63
:10081A00010E196F000E1A6F57DE15C2E1FF16C2DC
:10082A00E2FF00C0E6FF13C215F214C216F2010E6F
:10083A000201196F000E1A6F47DE15C2E1FF16C2D8
:10084A00E2FF00C0E6FF0201196B1A6B3DDE5CDCB9
:10085A000FC207F210C208F211C209F212C20AF25A
:02086A0012007A
:10086C00819A819481888184819481888184819406
:10087C0002010FA502D0818801D0819881848194D6
:10088C000FA302D0818801D08198818481940FA11B
:10089C0002D0818801D0819881848194819881844F
:1008AC008194818481948184046A056A000E026EAD
:1008BC00080E036E800E006E800E0318005C02E1C1
:1008CC00025001080EE2819481A604D00250042645
:1008DC0003500522818403320232039E03BC038E33
:0E08EC00E9D7818A04C000F005C001F01200B7
:1008FA009E0E0101F46F010EF56F190EF66F020ECE
:10090A00F76F560EF06F090EF16F000EF26F000EC0
:10091A00F36F6E0E0201016F050E026F000E036F78
:10092A00000E046FFF0E0101FA6FFF0EFB6F000E3F
:10093A00FC6F000EFD6FAC8A900EAB6E948E949C89
:0C094A009EAA03D0AECF00F0FBD7120035
:10095600AECFF9F1ABA202D0AB98AB88F9C100F0EB
:0209660012007D
:10096800C26AC00EC212C18CC18E0FC200F000361E
:10097800009000360090003600900050C212C280ED
:10098800A2EC00F0C284C2A401D0FDD7C4CF01F00C
:0E099800006AC3500012000E0112C29012003D
:1009A6000201156B166B000E165D02E10A0E155D4F
:1009B6000BE215511325E16E16511421E26E200E3D
:1009C600E66E154B162BEFD715511325E16E165112
:1009D6001421E26EE66A010E155F000E165B1551D4
:1009E6001325176F16511421186F0A0E046E000E88
:1009F600056E066E076E0FC200F010C201F011C23E
:100A060002F012C203F0F3EC00F008C000F009C0D7
:100A160001F00AC002F00BC003F0300E002617C228
:100A2600E1FF18C2E2FF00C0E6FF0A0E046E000EE8
:100A3600056E066E076E0FC200F010C201F011C2FD
:100A460002F012C203F0F3EC00F000C00FF201C096
:100A560010F202C011F203C012F2000E046E031867
:100A660008E10450021805E10450011802E10050A3
:100A7600000A01E105D0010E155F000E165BAFD727
:020A860012005C
:100A88008DEC08F0EEDD0F0EAF6EAC8432DFECC1FA
:100A98000FF2EDC110F2B90E0201116F000E126FC4
:100AA80010DE00C0ECF101C0EDF1EBDD80980D0E19
:100AB8000B6EAF0E0C6EB60E0D6E0D2EFED70C2EF5
:100AC800FCD70B2EFAD7000081800D0E0B6EAF0EEF
:100AD8000C6EB60E0D6E0D2EFED70C2EFCD70B2EFF
:100AE800FAD70000ECC10FF2EDC110F2910E116FB0
:100AF800000E126FE6DD00C0ECF101C0EDF1C1DDC2
:100B0800ECC10FF2EDC110F2510E116F000E126F11
:100B1800D8DD00C0ECF101C0EDF1B3DDECC10FF29E
:100B2800EDC110F2440E116F010E126FCADD00C044
:100B3800ECF101C0EDF1A5DDECC10FF2EDC110F251
:100B4800080E116F010E126FBCDD00C0ECF101C080
:100B5800EDF197DDECC10FF2EDC110F2CF0E116F80
:100B6800000E126FAEDD00C0ECF101C0EDF189DDC1
:100B7800ECC10FF2EDC110F2290E116F000E126FC9
:100B8800A0DD00C0ECF101C0EDF10101FF6B0C0E1E
:100B98000201006F066B8C0E056F8C0E0F6F000E36
:100BA800106F27C011F228C012F2E2DCECC10FF27C
:100BB800EDC110F227C011F228C012F222DD00C0E8
:100BC800ECF101C0EDF15DDDD3DD1A0E0B6E5E0EAA
:100BD8000C6E6E0E0D6E0D2EFED70C2EFCD70B2E46
:100BE800FAD7000002010D6B0E6B02010D4B0E2BA4
:100BF8000DC20FF20EC210F2ECC111F2EDC112F2E9
:100C0800B7DC3FDD090E196FCFEC00F0ECC10FF235
:100C1800EDC110F2150E0201116F000E126F51DDB9
:100C280000C0ECF101C0EDF12CDD0B6B0C6B800EFC
:100C38000C19006E800E005C02E1050E0B5D33E2BC
:100C48000BC20FF28DDE00C0EEF101C0EFF1ECC176
:100C58000FF2EDC110F24B0E0201116F000E126F70
:100C680030DD00C0ECF101C0EDF1020E0024E16EB0
:100C7800000E0120E26E300E0B25006E00C0E6FF6C
:100C880000DDEEC10FF2EFC110F2ECC111F2EDC1BF
:100C980012F26EDCF6DC090E196FCFEC00F00201DF
:100CA8000B4B0C2BC4D764DD090E0201196FCFEC76
:100CB80000F0ECC10FF2EDC110F2380E0201116F15
:100CC800000E126FFEDC00C0ECF101C0EDF1D9DCC2
:100CD8000B6B0C6B800E0C19006E800E005C02E131
:100CE800080E0B5D34E2ECC10FF2EDC110F2810E7B
:100CF800116F010E126FE5DC00C0ECF101C0EDF1DF
:100D0800020E0024E16E000E0120E26E0B51300F3E
:100D1800006E00C0E6FFB5DC0BC20FF20CC210F289
:100D2800A1DD00C0EEF101C0EFF100C00FF201C07B
:100D380010F2ECC111F2EDC112F21ADCA2DC090EBC
:100D4800196FCFEC00F002010B4B0C2BC3D710DD51
:100D5800090E0201196FCFEC00F0ECC10FF2EDC1E2
:100D680010F26E0E0201116F010E126FAADC00C0A4
:100D7800ECF101C0EDF185DC0B6B0C6B10D0200E93
:100D88000101FF6F26D00101400EFF6F22D0010143
:100D9800600EFF6F1ED00101FF6B1BD01AD0000E32
:100DA80002010C1902E1000E0B19E9E0000E0C1902
:100DB80002E1010E0B19E7E0000E0C1902E1020E28
:100DC8000B19E5E0000E0C1902E1030E0B19E3E024
:100DD800E5D70201ECC10FF2EDC110F2680E116FF8
:100DE800010E126F6EDC00C0ECF101C0EDF1020ED5
:100DF8000024E16E000E0120E26E300E0B25006E1D
:100E080000C0E6FF3EDCBDDC07C20FF208C210F2EC
:100E180009C211F20AC212F2ECC113F2EDC114F2C6
:100E2800BEDD2FDC090E196FCFEC00F0020E0B6E41
:100E3800450E0C6EA90E0D6E0D2EFED70C2EFCD78E
:100E48000B2EFAD70000000002010B4B0C2B800E72
:100E58000C19006E800E005C02E1040E0B5D8EE33F
:100E6800090E196FCFEC00F0ECC10FF2EDC110F2D2
:100E7800990E0201116F010E126F23DC00C0ECF114
:100E880001C0EDF1FEDB06C20FF2000E106FECC1DF
:100E980011F2EDC112F2BCEC02F045EC03F068DC93
:100EA800B7EC02F000523AE052DD00C0FEF100500B
:100EB8005A0803E2200E0101FE5F0D0E0201196FB0
:100EC800CFEC00F0ECC10FF2EDC110F2870E020179
:100ED800116F010E126F65EC03F000C0ECF101C058
:100EE800EDF145EC03F0FEC119F2CFEC00F0090E6C
:100EF8000201196FCFEC00F0FEC10FF209DC38DCFB
:100F0800070E0B6E580E0C6E590E0D6E0D2EFED779
:100F18000C2EFCD70B2EFAD700000000520E0C6ED8
:100F2800290E0D6E0D2EFED70C2EFCD700000000EA
:080F3800817080785AD6FFD7C2
:10111A0010EE15F0D90E006E020E016E400EF66E3C
:0E112A000F0EF76E000EF86EAFEC02F0120022
:100F400041444320313062697473202020202020E6
:020F50003A0065
:020F5200E001BC
:0F0F5400436F6E666967204144433138623D0048
:100F63004D43503333303420313262697473203A45
:030F73002020003B
:060F76004368303D20003D
:100F7C005473745F3138463235385F52532E6320C8
:100F8C0031322F31322F3230313020696E7465722C
:100F9C00666163652052533233322061766563207B
:100FAC0032205472616E736973746F72730A0D0020
:100FBC00417665632074696E79626C6431384632AF
:100FCC0035385F31304D687A5F3139323030626498
:080FDC00732E4845580A0D0070
:100FE400494E49542075736172742033383430305B
:060FF4006264730A0D00A7
:100FFA0054657374204F4B206475204D435033342D
:10100A0032342034434820313862697473202C65A5
:10101A006E206C696169736F6E2049324320536F89
:09102A006674776172650A0D001D
:1010330054657374204F4B206475204D43503330F7
:10104300342038206368616E656C7320313220620E
:101053006974732C206C696169736F6E20535049F6
:0C10630020736F6674776172650A0D00DF
:10106F0035206368616E656C7320414443313020D5
:10107F0062697473206475205049433138463235A4
:04108F00380A0D000E
:061093004348303D20003F
:101099004D43503334323420313862697473203A05
:0310A90020200004
:0610AC004348303D200026
:1010B2007265637520436172616374657265203A7B
:0210C20020000C
:0710C4004761696E3D200049
:1010CB0031323334353637383930313233343536D3
:1010DB0037383930313233343536373839303132BD
:1010EB0033343536373839303431323334353637AB
:1010FB0038393031323334353637383930313200D4
:0C110B003132343536373839303132009B
:02111700A00135
:020000040030CA
:0D000100220F0EFFFF81FF0FC00FE00F4028
:00000001FF
